:020000040800F2
:10000000882B00202502000829030008210300088E
:1000100025030008E1020008990300080000000021
:100020000000000000000000000000003103000894
:10003000E5020008000000002D0300083503000859
:100040003F0200083F0200083F0200083F0200088C
:100050003F0200083F020008E90200083F020008D2
:100060003F0200083F0200083F0200083F0200086C
:100070003F0200083F0200083F0200083F0200085C
:100080003F0200083F0200083F0200083F0200084C
:100090003F0200083F0200083F0200083F0200083C
:1000A0003F0200083F0200083F0200083F0200082C
:1000B0003F0200083F0200083F0200083F0200081C
:1000C0003F0200083F0200083F0200083F0200080C
:1000D0003F0200083F0200083F0200083F020008FC
:1000E0003F0200083F0200083F0200083F020008EC
:1000F0003F0200083F0200083F0200083F020008DC
:100100003F0200083F0200083F0200083F020008CB
:100110003F0200083F0200083F0200083F020008BB
:100120003F0200083F0200083F0200083F020008AB
:100130003F0200083F0200083F0200083F0200089B
:1001400000000000000000000000000000000000AF
:100150003F0200083F0200083F0200083F0200087B
:100160003F0200083F0200083F0200083F0200086B
:100170003F0200083F0200083F0200083F0200085B
:100180003F02000800F002F800F03CF80AA090E8F6
:10019000000C82448344AAF10107DA4501D100F042
:1001A00031F8AFF2090EBAE80F0013F0010F18BFD3
:1001B000FB1A43F00103184788470000A8470000D6
:1001C000103A24BF78C878C1FAD8520724BF30C883
:1001D00030C144BF04680C60704700000023002455
:1001E00000250026103A28BF78C1FBD8520728BF47
:1001F00030C148BF0B6070471FB501F0CFFE1FBD77
:1002000010B510BD00F031F81146FFF7F5FF01F011
:100210007FFC00F04FF803B4FFF7F2FF03BC00F0DF
:1002200057F800000948804709480047FEE7FEE705
:10023000FEE7FEE7FEE7FEE7FEE7FEE7FEE7FEE796
:1002400004480549054A064B704700003903000879
:100250008501000888250020882B002088270020A1
:1002600088270020704770477047754600F02CF8CB
:10027000AE4605006946534620F00700854618B093
:1002800020B5FFF7DDFFBDE820404FF000064FF03E
:1002900000074FF000084FF0000BAC46ACE8C00977
:1002A000ACE8C009ACE8C009ACE8C00921F007011E
:1002B0008D46704710B50446AFF300802046BDE878
:1002C0001040FFF7A8BF000000487047080000205A
:1002D00001491820ABBEFEE726000200704700006F
:1002E000FEE700007047000080B5052000F0D2F95D
:1002F000012001F0E9FA40F60000C4F201000121FA
:1003000001F0D6FB002818BF80BD40F20000C2F209
:10031000000001780422042908BF0122027080BD78
:10032000FEE70000FEE70000704700007047000095
:1003300070470000704700004EF6885CCEF2000C5B
:10034000DCF8002041F2000142F47002C4F2020124
:10035000CCF800200A6842F001020A600A6892079D
:10036000FCD54A6822F003024A6000BF4A6812F0D6
:100370000C0FFBD100224A600B684FF6FF70CFF6DE
:10038000F260184008604FF41F000A6388604FF065
:1003900000604CF8800C7047FEE7000070B584B038
:1003A0004FF4C0100121012500F0DCF800200021ED
:1003B000002601F0D7FA01AC204601F07FFA40F2A6
:1003C0000110ADF80C0020468DF80460029501F094
:1003D00081FA032001F0A4FC06200021002201F094
:1003E00065FC04B070BD0000B0B582B00220C0F260
:1003F00018000121012500F0B5F86C46204601F0F7
:10040000A7FA41F60000C0F20010CDE9005040F616
:100410000000C4F20100214601F0EAFA02B0B0BDCA
:1004200041F20401C4F202010A6800F00F0022F058
:10043000F00242EA001008607047000041F2040137
:10044000C4F202010A6800F0070022F4E06242EA06
:10045000002008607047000041F20401C4F202016C
:100460000A6800F0070022F4605242EAC0200860E7
:100470007047000041F25401C4F202010A680128E9
:1004800022F0300208BF30320A607047042888BF6B
:100490007047DFE800F0030C19262F0041F200003E
:1004A000C4F20200026861F300020260704741F288
:1004B0000000C4F20200026801F0010122F480325F
:1004C00042EA01410160704741F20000C4F20200BB
:1004D000026801F0010122F0807242EA01610160CC
:1004E000704741F20000C4F20200026A61F30002A8
:1004F0000262704741F20000C4F20200426A61F3F6
:10050000000242627047000041F20002010CC4F296
:100510000202895800F01F0021FA00F000F00100EB
:100520007047000041F25401C4F202010A6800F071
:10053000030022F4405242EA003008607047000095
:1005400041F200010020C4F2020100BF0A689203D8
:1005500004D4B0F5405F00F10100F7D30868C0F3A0
:100560004040704741F2000200F01F034FF0010CC1
:10057000C4F2020201290CFA03F14FEA1040835839
:1005800014BF23EA010119438150704780B541F23D
:10059000040EC4F2020EDEF800C060B14CF48033E9
:1005A000CEF80030DEF800C0012814BF4CF4003053
:1005B0002CF4003001E02CF48030CEF80000DEF89E
:1005C000000061F39540CEF80000DEF80000090954
:1005D00061F35E70CEF80000DEF8000020F000400D
:1005E00040EAC270CEF8000080BD000041F2000079
:1005F000C4F20200016841F001010160016889074D
:10060000FCD5416821F00301416000BF416811F051
:100610000C0FFBD10021416002684FF6FF73CFF64B
:10062000F2631A40026001634FF41F01816070475A
:1006300041F20401C4F202010A6860F301020A6097
:100640007047000041F20400C4F202000068C0F3E9
:100650008100704780B5042001F094FC40F2040052
:10066000C2F2000000684DF68361C4F21B31A0FBAA
:100670000101880C40F28401C2F2000108600868A0
:100680004FF47A71484340F28001C2F200010860E1
:1006900080BD000080B5002808BF80BD4EF210016B
:1006A00040F2800ECEF20001C2F2000E4FF0320C8A
:1006B000002300BF82B2332A06D3DEF8002032388E
:1006C00002FB0CF24A6004E0DEF800005043486090
:1006D00000208B600A6842F001020A600A6802F09A
:1006E0000112012AFAD00A6822F001020A6002040B
:1006F0008B60DFD180BD00002DE9F04381B08946D9
:10070000074640F6004800200021C4F2010800F02E
:10071000D7FF40464FF4804101F016F940464FF4B0
:10072000805101F011F9A8F554463046242101F01A
:1007300019FB00BF3046802101F016FB0028F9D1DB
:1007400040464FF4805101F001F940464FF480419A
:1007500001F0FCF840464FF4805101F0F5F8002517
:100760007C5D00BF3046022101F0FEFA0028F9D07E
:100770003046214601F0F6FA0135B5F5945FEFD128
:100780003046802101F0F0FA0028F9D140464FF4BC
:10079000805101F0DBF80020002100F091FF40467D
:1007A0004FF4804101F0D0F840464FF4805101F001
:1007B000CBF83046262101F0D5FA00BF3046802123
:1007C00001F0D2FA0028F9D140464FF4805101F0EF
:1007D000BDF840464FF4804101F0B8F840464FF470
:1007E000805101F0B1F8002419F80450304602217C
:1007F00001F0BAFA0028F9D085F0FF01304601F087
:10080000B1FA0134B4F5945FEED100BF30468021D7
:1008100001F0AAFA0028F9D140464FF4805101F0C6
:1008200095F801B0BDE8F04300F0D6BF70B540F6D2
:1008300000440546C4F2010400F05AFE20464FF47D
:10084000804101F081F820464FF4805101F07CF89E
:10085000A4F554463046102101F084FA3046802138
:1008600001F082FA0028F9D120464FF4805101F0BE
:100870006DF820464FF4804101F068F820464FF4AF
:10088000805101F061F83046294601F06BFA00BF53
:100890003046802101F068FA0028F9D120464FF453
:1008A000805101F053F840F27C00C2F200000021B8
:1008B000017070BDF0B581B040F27C06C2F2000656
:1008C000307840F60044C4F2010498B9A4F580657C
:1008D00028464FF4807101F037F83220FFF7DAFE36
:1008E00028464FF4807101F031F83220FFF7D2FE34
:1008F00001203070A4F5806630464FF4007101F09D
:10090000D7F870B149F641450120013D00F044821D
:10091000FFF7C0FE30464FF4007101F0C9F800281F
:10092000F2D120464FF4804101F00EF820464FF4FA
:10093000805101F009F8A4F554452846122101F030
:1009400011FA00BF2846802101F00EFA0028F9D1E3
:1009500020464FF4805100F0F9FF20464FF48041CB
:1009600000F0F4FF0A20FFF795FE30464FF40071C7
:1009700001F09EF878B149F6414700BF0120013FE0
:1009800000F00A82FFF786FE30464FF4007101F056
:100990008FF80028F2D120464FF4804100F0D4FFB8
:1009A00020464FF4805100F0CFFF2846012101F08E
:1009B000D9F900BF2846802101F0D6F90028F9D1E5
:1009C00020464FF4805100F0C1FF20464FF4804193
:1009D00000F0BCFF20464FF4805100F0B5FF2846E0
:1009E000272101F0BFF900BF2846802101F0BCF9A2
:1009F0000028F9D120464FF4805100F0A7FF20468F
:100A00004FF4805100F0A0FF2846012101F0AAF91F
:100A10002846802101F0A8F90028F9D120464FF49A
:100A2000805100F093FF20464FF4805100F08CFF7E
:100A30002846012101F096F92846802101F094F919
:100A40000028F9D120464FF4805100F07FFF204666
:100A50004FF4804100F078FF20464FF4805100F0C1
:100A600073FF2846112101F07DF900BF284680213F
:100A700001F07AF90028F9D120464FF4805100F0B6
:100A800065FF20464FF4804100F060FF20464FF4A0
:100A9000805100F059FF2846012101F063F900BFA1
:100AA0002846802101F060F90028F9D120464FF452
:100AB000805100F04BFF20464FF4804100F044FF8E
:100AC00020464FF4805100F03FFF2846442101F0BA
:100AD00049F900BF2846802101F046F90028F9D1E4
:100AE00020464FF4805100F031FF20464FF4804102
:100AF00000F02CFF20464FF4805100F025FF2846DF
:100B0000002101F02FF900BF2846802101F02CF9C7
:100B10000028F9D120464FF4805100F017FF2046FD
:100B20004FF4805100F010FF28460F2101F01AF910
:100B30002846802101F018F90028F9D120464FF409
:100B4000805100F003FF20464FF4804100F0FCFE8E
:100B500020464FF4805100F0F7FE2846452101F071
:100B600001F900BF2846802101F0FEF80028F9D1E4
:100B700020464FF4805100F0E9FE20464FF48041BA
:100B800000F0E4FE20464FF4805100F0DDFE2846E0
:100B9000272101F0E7F800BF2846802101F0E4F8A2
:100BA0000028F9D120464FF4805100F0CFFE2046B6
:100BB0004FF4805100F0C8FE2846012101F0D2F820
:100BC0002846802101F0D0F80028F9D120464FF4C2
:100BD000805100F0BBFE20464FF4805100F0B4FE7F
:100BE0002846002101F0BEF82846802101F0BCF81B
:100BF0000028F9D120464FF4805100F0A7FE20468E
:100C00004FF4805100F0A0FE2846002101F0AAF820
:100C10002846802101F0A8F80028F9D120464FF499
:100C2000805100F093FE20464FF4804100F08CFE8E
:100C300020464FF4805100F087FE28463C2101F009
:100C400091F800BF2846802101F08EF80028F9D1E4
:100C500020464FF4805100F079FE20464FF4804149
:100C600000F074FE20464FF4805100F06DFE2846DF
:100C7000052101F077F800BF2846802101F074F8C3
:100C80000028F9D120464FF4805100F05FFE204645
:100C90004FF4804100F058FE20464FF4805100F0A0
:100CA00053FE2846212101F05DF800BF284680212F
:100CB00001F05AF80028F9D120464FF4805100F095
:100CC00045FE20464FF4804100F040FE20464FF4A0
:100CD000805100F039FE2846002101F043F800BFA2
:100CE0002846802101F040F80028F9D120464FF431
:100CF000805100F02BFE20464FF4805100F024FE7E
:100D00002846802101F02EF82846802101F02CF899
:100D10000028F9D120464FF4805100F017FE2046FC
:100D20004FF4804100F010FE20464FF4805100F057
:100D30000BFE2846182101F015F800BF2846802137
:100D400001F012F80028F9D120464FF4805100F04C
:100D5000FDFD20464FF4804100F0F8FD20464FF4A1
:100D6000805100F0F1FD2846802100F0FBFF00BF1C
:100D70002846802100F0F8FF0028F9D120464FF4E2
:100D8000805100F0E3FD0020002100F099FC00F00C
:100D900023FC002818BF012001B0F0BD2DE9F0416F
:100DA00084B00224C0F2180420460121FFF7DAFBC8
:100DB000601C0121FFF7D6FB02AD284600F0C8FDFC
:100DC00040F60044C4F20104A4F5806630464FF4B6
:100DD00080714FF4807700F0B7FD40F20040C0F220
:100DE0001010CDE902703046294600F001FE1820AF
:100DF000ADF80D004FF4007002903046294600F027
:100E0000F7FD20464FF480414FF4804600F09EFDF0
:100E10004FF010084FF48067204629468DF80E8069
:100E2000ADF80C70029600F0E3FD4FF40050082678
:100E3000029020462946ADF80C708DF80E6000F047
:100E4000D7FD4FF400400290204629468DF80E60F1
:100E500000F0CEFD20464FF480514FF4805600F054
:100E600075FD204629468DF80E80ADF80C7002966F
:100E700000F0BEFD0E20C0F21C000121FFF772FB46
:100E80006D46284600F05CFF40F20310C0F20500FA
:100E9000009040F20010C0F20110A4F554440190FB
:100EA0002046294600F066FF2046012100F050FF51
:100EB00004B0BDE8F081000080B540F2680CC2F2D9
:100EC000000CBCF81210002908BF80BD4FF0000EC6
:100ED00006E000BFBCF812100EF1010E8E4512D2D2
:100EE000BCF81030002BF5D04FF0FF31DCF80020BB
:100EF0000EFB03220A445070BCF810308A1C0131EA
:100F00009A42F3D3E6E780BD2DE9F04F86B0B2EB0D
:100F1000000C0D46924648BFCCF1000C5F1B4FF011
:100F2000FF314FF6FF7248BF7F424FF0FF368245D8
:100F300088BF0121029119460193AB4288BF012667
:100F400040F26809A2F18003C7F1000B0096ACEBF8
:100F50000706C2F200090FFA83FE0397691E049583
:100F6000059102E0BCEB460F4CDAB9F80E30A0F167
:100F70000108B32B0CDC9BB15A2B38D1B9F80830DF
:100F8000B9F80A700499A3EB00087B1A17E000BFB8
:100F9000B42B0FD0B3F5877F059B10D027E000BF9F
:100FA0005146B9F808A0049A4346AAEB02088A46BB
:100FB00005E000BFB9F80A30DDF814801B1AB9F853
:100FC00010209BB21FFA88F75A43D9F8003002EB81
:100FD000D7029F5C08F007058021E9400F9C394348
:100FE0004EFA05F5002C08BF07EA05019954BBEB42
:100FF000460FB7DC81B251450ED00399761A02999B
:101000000844AFE70499019A89B2914204D0049D43
:10101000009966440D44A1E706B0BDE8F08F0000DA
:101020002DE9F04182B00F46DDE908811C461546E6
:10103000064681B1A7420BD2B9B230462A460B46CA
:10104000CDF80080FFF760FF0137B8B2A042F3D3BC
:1010500002B0BDE8F081304639462A463B46CDF81D
:101060000080FFF751FF3046394632462346CDF81F
:101070000080FFF749FF284621462A463B46CDF827
:101080000080FFF741FF2846214632462346CDF82F
:101090000080FFF739FF02B0BDE8F08110B540F2E3
:1010A000680EDDF808C0C2F2000ECEF80000C808D5
:1010B000AEF80810AEF80A20AEF80CC04FF0010CE4
:1010C0004C0718BF0CEBD100AEF81000AEF80E3094
:1010D000B3FA83F0B43BB3FA83F340095B091843D6
:1010E0000846AEF812201CBF10460A46AEF80400AF
:1010F000AEF8062010BD000040F26801C2F2000107
:10110000086070472DE9F04F8BB00130069080B237
:101110000590C01AB0F5947F00F3EF80082B02D140
:1011200006276FB9E9E0D8085F074FF0010618BF3E
:1011300006EBD3005F08784387B2002F00F0DD8014
:10114000A2F1200085B25808039041F6B67005EB75
:101150004502C0F6000000EB4200049042F25260EB
:1011600040F26806C0F60000DDF818E001314FF6E5
:101170007F7B00240192C2F20006802200EB051062
:1011800002950090CDE9077312E000BF05991FFAA0
:101190008EF0401A03998842069808BF864609993E
:1011A00008BF083107980A9C0134844200F0A580EA
:1011B000082B0A9402D1049818E000BF182B0AD01B
:1011C000102B12D00C2B40F09880019842F2DE13C5
:1011D000C0F6000306E0029842F6424300EBC0006E
:1011E000C0F6000303EB800000E00098204490F874
:1011F0000090AEF101084FF0000C099124E07089D5
:10120000A0EB0E00348A80B21FFA8AF36043346880
:1012100000EBD303E018E35C0AF007050FFA8BF745
:1012200022FA05F447FA05F51C4303EA0507149B67
:10123000002B08BF274607704FEA59090131BCF15E
:10124000070F0CF1010C4FD2F0895FEAC974A1F1CC
:10125000010A0BD1B32815DC20B35A28ECD1308910
:101260007389A0EB0E0A581ACCE700BFB32811DC33
:10127000E8B15A28E0D130897489A0EB0E0A601ACF
:101280001DE000BFB428BAD0B0F5877F5046C246F3
:10129000B8D0D1E7B4280FD0B0F5877F5046C2460A
:1012A0000DD0C9E73089A0EB010A4046AAE7308992
:1012B000A0EB010A404602E07089A0EB0E00378ADD
:1012C00080B21FFA8AF47843376800EBD4043819E7
:1012D0003C5D0AF007030FFA8BF522FA03F745FA93
:1012E00003F327431C40A2E7089B0EF1010E082BD5
:1012F0007FF44CAF0798099955E70BB0BDE8F08F24
:101300002DE9F04F89B0DE085F0705924FF001022A
:1013100018BF02EBD306002E009600F0BB80013010
:10132000DDF84C904E1C81B240F268070391002515
:10133000C2F200074FF0800C0024314604900AE00E
:101340000599019C029D0C4431460135009BAAB2CF
:101350009A4280F09F80059A002AF6D000230295D9
:10136000019413E00130039A81B2891A059A069C10
:101370009142049908BF0846089E08BF0836079B9B
:101380000134013399B291423146D9D2CDE90643B5
:10139000129BA2B213F80280A0F1010B4FF0000AD9
:1013A000089623E07A89121A3C8A92B21FFA8EF3C9
:1013B00062433C6802EBD302A518A35C4FF67F742E
:1013C0000EF0070624B22CFA06F244FA06F61A4387
:1013D0003340B9F1000F08BF1A462A704FEA580887
:1013E0000131BAF1070F0AF1010ABBD2FD895FEAA8
:1013F000C872A1F1010E0BD1B32D15DC25B35A2D06
:10140000ECD13A897B89A2EB000E5A1ACCE700BFD7
:10141000B32D11DCEDB15A2DE0D13A897B89A2EBD5
:10142000000E5A1A1CE000BFB42DBBD0B5F5877F63
:101430007246DE46B8D0D1E7B42D0FD0B5F5877F20
:101440007246DE460CD0C9E73A89A2EB010E5A4635
:10145000AAE73A89A2EB010E5A4601E07A89121AEC
:101460003D8A92B21FFA8EF36A434C46D7F8009039
:1014700002EBD3024FF67F7609EB020519F8022042
:10148000A1460EF0070436B22CFA04F326411343AA
:1014900032409EE709B0BDE8F08F00002DE9F0472B
:1014A00082B01C461378FBB1DDF828804FEA540A5D
:1014B0000D460646CAF59479571C06E05644B0B26C
:1014C000814511DB17F8013B73B1B0B2DAB229469E
:1014D0002346CDF80080FFF715FE082CEED1063626
:1014E000B0B2B0F5917FEDD902B0BDE8F087000051
:1014F000B0B540F60044C4F2010420464FF48041E8
:1015000000F022FA20464FF4805100F01DFAA4F5B5
:1015100054452846222100F025FC00BF28468021A2
:1015200000F022FC0028F9D120464FF4805100F051
:101530000DFA20464FF4804100F008FA20464FF49F
:10154000805100F001FA2846832100F00BFC00BF17
:101550002846802100F008FC0028F9D120464FF4ED
:10156000805100F0F3F920464FF4804100F0ECF98F
:1015700020464FF4805100F0E7F92846202100F082
:10158000F1FB00BF2846802100F0EEFB0028F9D1D6
:1015900020464FF4805100F0D9F920464FF48041A5
:1015A00000F0D4F9A4F5806420464FF4007100F0F7
:1015B0007FFA70B149F641450120013D08BFB0BD39
:1015C000FFF768F820464FF4007100F071FA002828
:1015D000F2D10020B0BD0000B0B540F60044C4F226
:1015E000010420464FF4804100F0AEF920464FF44C
:1015F000805100F0A9F9A4F554452846222100F0B5
:10160000B1FB00BF2846802100F0AEFB0028F9D1D5
:1016100020464FF4805100F099F920464FF4804164
:1016200000F094F920464FF4805100F08DF92846DF
:10163000F82100F097FB00BF2846802100F094FBC2
:101640000028F9D120464FF4805100F07FF9204660
:101650004FF4804100F078F920464FF4805100F0BB
:1016600073F92846202100F07DFB00BF2846802129
:1016700000F07AFB0028F9D120464FF4805100F0A9
:1016800065F920464FF4804100F060F9A4F58064CC
:1016900020464FF4007100F00BFA70B149F6414555
:1016A0000120013D08BFB0BDFEF7F4FF20464FF416
:1016B000007100F0FDF90028F2D10020B0BD00005B
:1016C000F0B581B040F60044C4F201040E46C708EC
:1016D00020464FF4804100F037F920464FF4805106
:1016E00000F032F9A4F5544528464E2100F03AFBAB
:1016F0002846802100F038FB0028F9D120464FF41D
:10170000805100F023F920464FF4804100F01EF98B
:1017100020464FF4805100F017F9F9B2284600F046
:1017200021FB00BF2846802100F01EFB0028F9D1D4
:1017300020464FF4805100F009F920464FF48041D3
:1017400000F002F920464FF4805100F0FDF82846E1
:101750004F2100F007FB00BF2846802100F004FB6A
:101760000028F9D140F22710861B20464FF4805103
:1017700000F0ECF820464FF4804100F0E7F82046F6
:101780004FF4805100F0E0F8F1B2284600F0EAFA98
:101790002846802100F0E8FA0028F9D120464FF4CD
:1017A000805100F0D3F820464FF4805100F0CCF87F
:1017B000C6F30021284600F0D5FA00BF2846802154
:1017C00000F0D2FA0028F9D120464FF4805101B040
:1017D000BDE8F04000F0BAB8B0B540F60044C4F23D
:1017E000010420464FF4804100F0AEF820464FF44B
:1017F000805100F0A9F8A4F554452846222100F0B4
:10180000B1FA00BF2846802100F0AEFA0028F9D1D5
:1018100020464FF4805100F099F820464FF4804163
:1018200000F094F820464FF4805100F08DF82846DF
:10183000F72100F097FA00BF2846802100F094FAC3
:101840000028F9D120464FF4805100F07FF820465F
:101850004FF4804100F078F820464FF4805100F0BA
:1018600073F82846202100F07DFA00BF2846802129
:1018700000F07AFA0028F9D120464FF4805100F0A8
:1018800065F820464FF4804100F060F8A4F58064CC
:1018900020464FF4007100F00BF970B149F6414554
:1018A000013D08BFB0BD0120FEF7F4FE20464FF415
:1018B000007100F0FDF80028F2D1B0BD00214160B8
:1018C000012101810170704740F21441C4F201010D
:1018D0000860704740F20841C4F20101426851F8C3
:1018E000083C934341F8083C51F8043C934341F8C9
:1018F000043C437A002B08BF704703786FEA020C60
:101900002BB151F8043C134341F8043C04E051F876
:10191000083C134341F8083C0B6803EA0C030B60D6
:101920004B6803EA0C034B60007A012807D018B912
:1019300008681043086070470868104308604868EA
:101940001043486070470000416170470161704773
:1019500040F200424FF6FF71C0F20012C0E90012DF
:101960007047000080B58B08032B88BF80BD0C2218
:1019700002EA810E4FF00F0C02EB83010CFA0EF21B
:10198000DFE803F002290F1C0821C4F201010B68F3
:1019900000FA0EF023EA02020A600A6810430860A7
:1019A00080BD0821C4F201018B6800FA0EF023EA21
:1019B00002028A608A681043886080BD0821C4F2F0
:1019C0000101CB6800FA0EF023EA0202CA60CA687D
:1019D0001043C86080BD0821C4F201014B6800FAC1
:1019E0000EF023EA02024A604A681043486080BD54
:1019F000B0B58B790A88032B0BD07BB9497928299C
:101A000001F00F0E18D0182908BF0261110616D177
:101A10002EE04FF0000E110611D129E003F0080C62
:101A20000B79C97903F00403634401F0030103EB6C
:101A3000010E110603D11BE04261110618D00023EC
:101A40004FF00F0C002104E00131082903F10403D9
:101A50000ED022FA01F4E407F6D004680CFA03F57C
:101A6000AC43046004680EFA03F52C430460EBE712
:101A7000B2F5807F38BFB0BD120A00234FF00F0CC3
:101A8000002104E00131082903F104030ED022FAF9
:101A900001F4E407F6D044680CFA03F5AC43446063
:101AA00044680EFA03F52C434460EBE7B0BD000038
:101AB00080680840401AB0FA80F040097047000082
:101AC00010B582B00420C0F218000121FEF74AFDD3
:101AD0006C462046FFF73CFF40F20040C0F2101079
:101AE00001904FF40050009041F20000C4F2010058
:101AF0002146FFF77DFF02B010BD000041F20C004F
:101B0000C4F20100016881F40051016070470000D7
:101B100088B000F0A5F9FEF79DFDFEF765FCFEF725
:101B20003DFCFFF7CDFFFFF739F9FEF7C3FE40F2AA
:101B30008804C2F20004FF26204680214FF49472EC
:101B4000B4230096FFF7AAFA41F20835C2F2000565
:101B5000284680214FF49472B4230096FFF79EFA32
:101B60002046FFF7C9FAFF20FFF7A6F92846FFF73E
:101B7000C3FAFF20FFF7A0F943F69E10C0F600005D
:101B8000009017200321FA227A230196FFF7B8FB71
:101B900020462946FEF7B0FD01200126FEF746FE4D
:101BA0004FF4FA50FEF776FDFEF784FE2046FFF76D
:101BB000A3FAFF20FFF780F9002729A20A200021BD
:101BC00018230097FFF76AFC2AA20A20322110236B
:101BD0000097FFF763FC2EA20A201D211023009717
:101BE000FFF75CFC2846FFF787FAFF20FFF764F950
:101BF00046F26C40C0F22E00069045F22070C7F20B
:101C00006F20059046F66540C6F66C70049043F66A
:101C10003E60C4F62000039003AA0A20472118233F
:101C20000097FFF73BFC0A2067214FF48F72742363
:101C300000970196FFF7F4F920462946FEF75CFD70
:101C40000120FEF7F3FD40F20004C2F20004642517
:101C5000FFF754FF20786843FEF71CFDF8E700BF4C
:101C6000322E3920457061706572204D6F64756C3D
:101C70006500000077697468203239362078203199
:101C80003238207265736F6C7574696F6E00000076
:101C900044657369676E65642042792057654163C6
:101CA000742053747564696F00000000B0B54EF67F
:101CB0000C5ECEF2000EDEF800304FF0FF35C3F3BD
:101CC000022383F00704042C28BF0424033B05FAF5
:101CD00004F438BF0023A143994005FA03F39A4363
:101CE00000F00F03043B4EF2001C7344CEF2000CD4
:101CF00011430C33B0F1FF3F4FEA011100EB0C022E
:101D0000C8BF02F540730028197048BFB0BD00F08D
:101D10001F01012202FA01F140094CF82010B0BD68
:101D20004EF60C51CEF200010A684FF6FF031A403E
:101D300060F30A2242F0806040F0FD700860704756
:101D40000021C0F8031001600121C171704700003B
:101D5000026801F0010122F0400242EA81110160B3
:101D600070470000C16070478068084018BF0120BC
:101D700070470000C26922F40062C2610A78032A37
:101D800027D8DFE802F00206121A026822F40042A5
:101D90000EE0026822F400420260026822F48042EF
:101DA0000260026842F4806212E0026842F400427B
:101DB0000260026822F4804206E0026842F40042B7
:101DC0000260026842F480420260026822F480628B
:101DD0000260CA79036802F0010223F4007343EA47
:101DE000422202604A78012A06D1CA79012A03D127
:101DF000026842F4807202E0026822F4807202609B
:101E00004A78036862F3820303608A784368072A8A
:101E100023F4807388BF03F5807343608A78036876
:101E200062F3C5030360CA78036802F0010223F07D
:101E3000800343EAC21202600A79036802F00102D9
:101E400023F4006343EAC22202604A79036862F322
:101E5000410303608979026861F300020260704700
:101E600080B5FEF7C3FB01200121FEF70FFB00BF89
:101E7000FEF766FB0028FBD002203B210122FEF783
:101E800085FB0020FEF74EFB02200121FEF7FEFA43
:101E90001920FEF739FB0128FAD10020FEF7C0FA1D
:101EA0000420FEF7D9FA0420FEF7C8FA0120FEF755
:101EB000E1FA0220FEF7BCFBFEF7C4FB0228FBD1CF
:101EC0000020FEF7D7FABDE8804000F001B800001E
:101ED000B0B541F2040441F20025C4F20204C0F29C
:101EE0007A05FEF7AFFB02280BD0A0BB206D800562
:101EF00031D5E06A800144BF46F60045C0F2DC25DA
:101F000029E0D4F800C021682268C1F38341C2F3FC
:101F100041721301581C0F29034618BF0223002ADF
:101F200018BF03465FEACC3003EB010006D440F64D
:101F30000011C0F23D0100FB01F50CE021688903AE
:101F400001D4454307E0216DC1F301310231B5FBF6
:101F5000F1F101FB00F540F20400C2F2000005605F
:101F6000216804A2C1F30311515C026822FA01F155
:101F70000160B0BD00000000000000000102030489
:101F8000060708094EF21001CEF200010A68042883
:101F900022F0040208BF04320A607047F1EE100A12
:101FA0004FF6FF71C0F2C03120EA010040F04070EE
:101FB000E1EE100A70470000000000000000002F52
:101FC000000000000700070000147F147F140024A5
:101FD0002A7F2A12006264081323003649552250D2
:101FE00000000503000000001C2241000000412207
:101FF0001C000014083E08140008083E08080000F1
:1020000000A06000000808080808000060600000E8
:10201000002010080402003E5149453E0000427F66
:102020004000004261514946002141454B310018B2
:1020300014127F10002745454539003C4A49493074
:10204000000171090503003649494936000649492E
:10205000291E000036360000000056360000000839
:102060001422410000141414141400004122140816
:1020700000020151090600324959513E007C1211FB
:10208000127C007F49494936003E41414122007F90
:102090004141221C007F49494941007F090909014A
:1020A000003E4149497A007F0808087F0000417FCF
:1020B0004100002040413F01007F08142241007F81
:1020C00040404040007F020C027F007F0408107FE8
:1020D000003E4141413E007F09090906003E415151
:1020E000215E007F0919294600464949493100010E
:1020F000017F0101003F4040403F001F2040201F62
:10210000003F4038403F0063140814630007087024
:10211000080700615149454300007F4141000055D7
:102120002A552A55000041417F00000402010204A3
:102130000040404040400000010204000020545490
:102140005478007F484444380038444444200038E0
:102150004444487F00385454541800087E09010252
:102160000018A4A4A47C007F080404780000447D27
:102170004000004080847D00007F10284400000063
:10218000417F4000007C04180478007C0804047837
:1021900000384444443800FC242424180018242423
:1021A00018FC007C0804040800485454542000041F
:1021B0003F444020003C4040207C001C2040201C2C
:1021C000003C4030403C004428102844001CA0A0A3
:1021D000A07C004464544C441414141414140000DF
:1021E000000000000000000000000000FC000000F3
:1021F000000002000000000C020C020000000000C1
:10220000000090D0BCD0BC90000300030000182454
:10221000FE448C000302070201001824D8B04C8051
:10222000000300010201C038E438E00001020201AD
:10223000020208060000000000000000000000008C
:1022400000F80402000000010204000204F800008B
:102250000004020100009060F8609000000001009E
:1022600000002020FC2020000000010000000000F1
:1022700000000000080600000000202020202000B0
:10228000000000000000000000000000000200004C
:1022900000000080601C0200040300000000F8043D
:1022A0000404F8000102020201000008FC00000022
:1022B00000020302000018844424180003020202F2
:1022C000020008042424D80001020202010040B0E8
:1022D00088FC80000000000302003C242424C40089
:1022E000010202020100F824242CC00001020202B3
:1022F00001000C04E41C0400000003000000D824CA
:102300002424D80001020202010038444444F800A9
:1023100000030202010000001000000000000200A3
:102320000000000020000000000006000000002067
:1023300050880402000000000102909090909000EC
:10234000000000000000000204885020000201008C
:1023500000001804C4241800000002000000F80463
:10236000E494F80001020202020000E09CF0800008
:1023700002030000030204FC2424D800020302022A
:102380000100F80404040C0001020202010004FC34
:102390000404F80002030202010004FC24740C008F
:1023A00002030202030004FC24740C000203020076
:1023B0000000F0080444CC4000010202010004FCCB
:1023C0002020FC040203000003020404FC040400B7
:1023D000020203020200000404FC040406040403D5
:1023E000000004FC24D00C0402030200030204FCDD
:1023F00004000000020302020203FC3CC03CFC009B
:1024000003000300030004FC30C4FC0402030200C8
:102410000300F8040404F80001020202010004FCB5
:1024200024241800020302000000F8848404F80049
:1024300001020207050004FC246498000203020064
:102440000302182424448C000302020201000C043D
:10245000FC040C0000020302000004FC0000FC0469
:10246000000102020100047C80E01C040000030063
:1024700000001CE03CE01C00000300030000049C82
:10248000609C0400020300030200041CE01C040022
:102490000002030200000C84641C04000203020218
:1024A00003000000FE020200000007040400000E0A
:1024B00030C00000000000010200000202FE000027
:1024C00000040407000000040204000000000000F3
:1024D00000000000000000000808080808080000CC
:1024E000020000000000000000000040A0A0C000AA
:1024F00000010202030204FC2020C00000030202CB
:10250000010000C02020600000010202020000C0A3
:102510002024FC0000010202030200C0A0A0C000B1
:102520000001020202000020F82424040002030239
:1025300002000040A0A0602000070A0A0A0404FC70
:102540002020C0000203020003020020E40000007B
:10255000000203020000000020E400000808080751
:10256000000004FC80E020200203020003020404B7
:10257000FC000000020203020200E020E020C00094
:1025800003000300030020E02020C000020302003B
:10259000030200C02020C00000010202010020E070
:1025A0002020C000080F0A02010000C02020E00027
:1025B0000001020A0F0820E0402020000203020070
:1025C00000000060A0A02000000202020300002022
:1025D000F820000000000102020020E00020E000DE
:1025E00000010202030220E02080602000000301BD
:1025F00000006080E08060000003000300002060B5
:102600008060200002030003020020E020806020A0
:102610000808070100000020A0602000000203025B
:102620000200000020DE020000000007040000009D
:1026300000FF00000000000F00000002DE2000008C
:102640000004070000000201020404020000000070
:10265000000000000000000000000000000000007A
:102660000000000000F8000000000000003330000F
:10267000000000100C06100C060000000000000016
:10268000000040C07840C0784000043F04043F048C
:102690000400007088FC08300000001820FF211E94
:1026A0000000F008F000E018000000211C031E21CB
:1026B0001E0000F00888700000001E212324192746
:1026C000211010160E0000000000000000000000A5
:1026D0000000000000E018040200000000071820BD
:1026E000400000020418E00000000040201807002D
:1026F0000000404080F0804040000202010F0102D3
:102700000200000000F0000000000101011F0101B3
:102710000100000000000000000080B07000000018
:1027200000000000000000000000000101010101A4
:102730000101000000000000000000303000000037
:10274000000000000000806018040060180601000E
:10275000000000E010080810E000000F102020101A
:102760000F00001010F8000000000020203F202083
:10277000000000700808088870000030282422211A
:1027800030000030088888483000001820202011D0
:102790000E000000C02010F8000000070424243FB1
:1027A000240000F80888880808000019212020115A
:1027B0000E0000E0108888180000000F1120201182
:1027C0000E0000380808C83808000000003F00006C
:1027D00000000070880808887000001C2221212257
:1027E0001C0000E010080810E00000003122221157
:1027F0000F00000000C0C0000000000000303000EA
:102800000000000000800000000000008060000068
:1028100000000000804020100800000102040810A1
:1028200020004040404040404000040404040404B0
:10283000040000081020408000000020100804025E
:102840000100007048080808F00000000030360160
:102850000000C030C828E810E0000718272423141F
:102860000B000000C038E0000000203C23020227DB
:10287000382008F8888888700000203F2020201128
:102880000E00C03008080808380007182020201063
:10289000080008F808080810E000203F2020201059
:1028A0000F0008F88888E8081000203F2020232027
:1028B000180008F88888E8081000203F200003006E
:1028C0000000C03008080838000007182020221E29
:1028D000020008F808000008F808203F2101012143
:1028E0003F20000808F8080800000020203F2020B2
:1028F000000000000808F8080800C08080807F0001
:10290000000008F888C028180800203F2001263859
:10291000200008F8080000000000203F20202020B0
:10292000300008F8F800F8F80800203F003F003FAA
:10293000200008F830C00008F808203F20000718E1
:102940003F00E01008080810E0000F1020202010C1
:102950000F0008F808080808F000203F21010101D5
:102960000000E01008080810E0000F182424385078
:102970004F0008F8888888887000203F2000030CEA
:1029800030200070880808083800003820212122F3
:102990001C00180808F8080818000000203F200054
:1029A000000008F808000008F808001F2020202078
:1029B0001F000878880000C83808000007380E019A
:1029C0000000F80800F80008F800033C0700073C86
:1029D0000300081868808068180820302C03032C36
:1029E00030200838C800C83808000000203F200008
:1029F000000010080808C8380800203826212020C8
:102A00001800000000FE020202000000007F4040AB
:102A10004000000C30C0000000000000000106383B
:102A2000C00000020202FE000000004040407F00A3
:102A30000000000004020202040000000000000088
:102A40000000000000000000000080808080808086
:102A5000808000020204000000000000000000006E
:102A600000000000808080800000001924222222C3
:102A70003F2008F8008080000000003F1120201156
:102A80000E000000008080800000000E1120202039
:102A90001100000000808088F800000E1120201036
:102AA0003F200000808080800000001F2222222220
:102AB0001300008080F0888888180020203F2020A4
:102AC00000000000808080808000006B94949493CC
:102AD000600008F8008080800000203F2100002076
:102AE0003F2000809898000000000020203F202018
:102AF0000000000000809898000000C08080807F67
:102B0000000008F8000080808000203F24022D3063
:102B10002000000808F8000000000020203F2020CE
:102B200000008080808080808000203F20003F2047
:102B3000003F8080008080800000203F2100002036
:102B40003F200000808080800000001F2020202087
:102B50001F00808000808000000080FFA1202011E5
:102B60000E000000008080808000000E112020A058
:102B7000FF80808080008080800020203F21200016
:102B80000100000080808080800000332424242401
:102B90001900008080E0808000000000001F2020DD
:102BA00000008080000000808000001F2020201096
:102BB0003F20808080000080808000010E30080669
:102BC000010080800080008080800F300C030C307A
:102BD0000F0000808000808080000020312E0E31A8
:102BE0002000808080000080808080818E701806A8
:102BF000010000808080808080000021302C222114
:102C0000300000000000807C020200000000003F55
:102C1000404000000000FF00000000000000FF0036
:102C200000000002027C800000000040403F0000E5
:102C30000000000601010202040400000000000080
:102C40000000000000000000000000000000000084
:102C50000000000000000000000000000000000074
:102C60000000000000000000000000F0F0F0000094
:102C700000000000000000017F01000000000000D3
:102C80000000001C1C1C0000000000008060301CC4
:102C90008C60301C0C0000000000000000000000F0
:102CA0000000000000000000000000000000000024
:102CB00000E00000000000E000000086E69F86863D
:102CC0008686E69F860000011F01010101011F01A8
:102CD0000100000080C06020F820E0C0000000007B
:102CE00003070C18FF70E18100000000070F1010AF
:102CF0007F100F0700008060206080000000E0204F
:102D000000000F3020309F70DC371030C000000012
:102D1000100E03000718101807000000C02020E064
:102D2000C0000000000080E01F38E88703C43C04B6
:102D30000000070F1810100B070D1010080000807E
:102D40008C4C380000000000000000000000000073
:102D50000000000000000000000000000000000073
:102D6000000000000000000080E0300804000000C7
:102D7000000000FEFF010000000000000000000055
:102D8000030F1820400000040830E080000000001D
:102D900000000000000001FFFE00000000000040F5
:102DA00020180F03000000000000000000000000D9
:102DB000C00000000000004266663C18FF183C6638
:102DC0006642000000000000030000000000000058
:102DD0000000000080000000000000101010101023
:102DE000FF10101010100000000000000300000091
:102DF00000000000000000000000000000000000D3
:102E00000000000000000000000000808C4C380032
:102E100000000000000000000000000000000000B2
:102E20000000001010101010101010101000000002
:102E30000000000000000000000000000000000092
:102E40000000000000000000000000000000000082
:102E5000000000001C1C1C0000000000000000001E
:102E6000000000000000E0380C000000000080704E
:102E70001C03000000000060380E0100000000008C
:102E80000000000080C060202060C080000000FEC4
:102E9000FF010000000001FFFE000001070E1810F6
:102EA00010180E0701000000808080C0E0000000C4
:102EB00000000000000000FFFF0000000000000014
:102EC0001010101F1F101010000000804020202044
:102ED0002060C080000000030300804020381F07EE
:102EE0000000001C1A1918181818181F000000807C
:102EF000C020202060C080000000000303001010EC
:102F0000182FE780000000070F10101010180F078F
:102F10000000000000000000C0E0F000000000C061
:102F2000B088868180FFFF808000000000000010D4
:102F3000101F1F1010000000E060606060606060A3
:102F4000000000003F1008080818F0E0000000072B
:102F50000B101010101C0F030000000080C0402058
:102F60002020E0C0000000FCFF211008080818F035
:102F7000E0000001070C18101010080F03000000FB
:102F8000C0E06060606060E060000000030000007E
:102F9000E0180700000000000000001F1F000000F4
:102FA00000000080C0602020202060C080000087DA
:102FB000EF2C1818303068CF830000070F0810106E
:102FC0001010180F07000000C0C020202020C08073
:102FD0000000001F3F604040402010FFFE00000046
:102FE0000C1C101010080F0300000000000000006F
:102FF00000000000000000000000000E0E0E0000A7
:10300000000000000000001C1C1C0000000000006C
:103010000000000000000000000000000000000CA4
:103020000C00000000000000000000583800000004
:1030300000000000000000000080402010000000A0
:103040001028448201000000000000000000000081
:103050000102040810000000000000000000000051
:103060000000008484848484848484848400000038
:103070000000000000000000000000001020408060
:103080000000000000000000000000000182442851
:10309000100000001008040201000000000000C041
:1030A00020201010101030E0C0000003030000F0DA
:1030B00010080C070300000000001C1C1C0000008E
:1030C0000000000000C0406020202040C00000FC44
:1030D000FF01F00E03C1FE03807F0001070E0811FF
:1030E0001110110904020000000080E0E00000005F
:1030F00000000000807C4340477FF88000001018EB
:103100001F1000000000131F1C1020E0E0202020F2
:103110002060C080000000FFFF10101010182FE783
:103120008000101F1F1010101010180F0700000053
:1031300080C0402020202060E00000FCFF01000053
:103140000000000001000001070E18101010080414
:10315000030020E0E02020202040C080000000FF8D
:10316000FF000000000001FFFE00101F1F101010E4
:1031700018080E07010020E0E02020202020206019
:10318000800000FFFF101010107C00000000101FD6
:103190001F10101010101018060020E0E020202052
:1031A00020206060800000FFFF101010107C0000E5
:1031B0000100101F1F1000000000000000000000B0
:1031C00080C06020202040E0000000FCFF010000E3
:1031D0004040C0C140400001070E181010100F0FF2
:1031E000000020E0E0200000000020E0E02000FFE0
:1031F000FF101010101010FFFF00101F1F10000014
:103200000000101F1F100000202020E0E0202020E0
:1032100000000000000000FFFF00000000000000B0
:103220001010101F1F1010100000000000002020C0
:1032300020E0E020202000000000000000FFFF0050
:1032400000000060E0808080C07F3F00000020E040
:10325000E020000020A06020200000FFFF30187C4C
:10326000E3C000000000101F1F10000001131F1C0E
:10327000181020E0E020000000000000000000FF27
:10328000FF000000000000000000101F1F101010C1
:1032900010101018060020E0E0E000000000E0E060
:1032A000E02000FF013FFEC0E01E01FFFF00101FF5
:1032B0001000031F0300101F1F1020E0E0C00000DB
:1032C00000000020E02000FF0003071C78E08000E1
:1032D000FF00101F100000000000030F1F0000007F
:1032E00080C060202060C080000000FEFF01000060
:1032F000000000FFFE000001070E181010180C0758
:10330000010020E0E0202020202060C0800000FF9D
:10331000FF2020202020301F0F00101F1F10000052
:10332000000000000000000080C060202060C0801D
:10333000000000FEFF010000000000FFFE00000191
:10334000070E1111133C7C67210020E0E0202020B3
:10335000202060C0800000FFFF101030F0D0080F68
:103360000700101F1F10000000030F1C101000802A
:10337000C060202020204040E00000070F0C1818FB
:10338000303060E08100001F0C0810101010180F82
:1033900007008060202020E0E020202060800100E5
:1033A000000000FFFF000000000100000000101FEF
:1033B0001F100000000020E0E020000000000020BE
:1033C000E02000FFFF00000000000000FF000007F9
:1033D0000F1810101010100807002060E0E0200007
:1033E000000020E060200000077FF88000807C0360
:1033F000000000000000071F1C070000000020E084
:10340000E02000E0E0200020E0200007FFF8E01FBF
:10341000FFFCE01F00000000031F0300011F03006A
:103420000000002060E0A0000020E060200000001C
:1034300000038F7CF8C6010000000010181E130066
:1034400001171F1810002060E0E02000000020E0BD
:103450006020000001073EF8E018070000000000AF
:103460000010101F1F10100000000080602020209E
:1034700020A0E0E0200000000000C0F03E0F0300AC
:10348000000000101C1F171010101018060000007C
:10349000000000FC0404040404000000000000FF1D
:1034A00000000000000000000000007F404040409D
:1034B0004000000010E000000000000000000000DC
:1034C0000000031C608000000000000000000000FD
:1034D00000030C70800000000404040404FC0000DD
:1034E000000000000000000000FF000000000000DD
:1034F00040404040407F0000000000000010080CE9
:10350000040C081000000000000000000000000093
:1035100000000000000000000000000000000000AB
:10352000000000000000000000000000000000009B
:10353000000000000000808080808080808080808B
:103540008080000000040408080000000000000063
:10355000000000000000000000000000000000006B
:10356000000000000000000000000000000000005B
:103570000000000098D844642424FCF80000000FE8
:103580001F18101010081F1F10180020E0F0000076
:103590000000000000000000FFFF180804040CF801
:1035A000F00000001F0F18101010180F030000008B
:1035B0000000000000000000000000E0F818040413
:1035C000043C3800000000030F0C10101010080617
:1035D00000000000000000000020E0F0000000E01B
:1035E000F81C04040408FFFF000000030F1810106B
:1035F00010081F0F0800000000000000000000007D
:1036000000000000E0F8484444444C78700000009A
:10361000030F0C181010100804000000000080C0F8
:10362000602020E0C00000040404FFFF0404040440
:103630000000000010101F1F1010100000000000FC
:1036400000000000000000000000000070F88C0482
:10365000048CF874040C007076CF8D8D8D89C87839
:1036600070000020E0F000000000000000000000FA
:10367000FFFF08040404FCF8000000101F1F1000E6
:1036800000101F1F1000000000000060600000001C
:1036900000000000040404FCFC0000000000000026
:1036A0001010101F1F10101000000000000000007C
:1036B00000606000000000000000040404FCFC0046
:1036C00000000000C0C08080C07F3F0000000020DC
:1036D000E0F000000000000000000000FFFF80C0DC
:1036E000F41C0404000000101F1F1100031F1C1015
:1036F00010000000202020E0F0000000000000008A
:10370000000000FFFF000000000000001010101F6C
:103710001F1010100000000000000000000000005A
:10372000000004FCFC0804FCFC0804FCFC00101F66
:103730001F10001F1F10001F1F10000000000000BE
:103740000000000000000004FCFC08080404FCF871
:10375000000000101F1F100000101F1F10000000AD
:103760000000000000000000000000E0F0180C0461
:10377000040C18F0E00000030F0C101010100C0FD8
:103780000300000000000000000000000000000432
:10379000FCFC080404040CF8F0000080FFFF889093
:1037A00010101C0F030000000000000000000000CB
:1037B000000000E0F81C04040408F8FC000000030A
:1037C0000F1810109088FFFF80000000000000001C
:1037D000000000000000040404FCFC100804040CB9
:1037E0000C001010101F1F1010100000000000002F
:1037F0000000000000000000000000003078CCC491
:103800008484840C1C0000001E1810101011190F65
:1038100006000000000000C00000000000000004DE
:103820000404FFFF040404000000000000000F1F58
:103830001010100C0000000000000000000000004C
:1038400000000004FCFE00000004FCFE000000007C
:103850000F1F181010081F0F0800000000000000C4
:1038600000000000000000040C3CFCC40000C43C4C
:103870000C0400000000010F1E0E010000000000FB
:1038800000000000000000000000043CFCC400E454
:103890007CFC84807C040000071F070000071F07D2
:1038A0000000000000000000000000000000000414
:1038B000041C7CE4C0341C0404000010101C16011D
:1038C000131F1C1810000000000000000000000082
:1038D000000000040C3CFCC400C43C0404000000D4
:1038E000C080C1370E010000000000000000000091
:1038F00000000000000000001C0404C4F47C1C0450
:1039000000000000101C1F17111010180E000000FE
:103910000000000000F80C0400000000000000108F
:1039200028EF00000000000000000000003F6040A1
:103930000000000000000000FF0000000000000088
:1039400000000000FF000000000000000000000078
:10395000FF00000000000000040CF8000000000060
:10396000000000000000EF28100000000000000030
:1039700040603F0000000000000000180602020442
:1039800008102020300800000000000000000000A7
:103990000000000000000000000000000000000027
:1039A0000000000000000000000000000000000017
:1039B0000000000000000000000000000000000007
:1039C00000000000000000000000000000000000F7
:103F40000000000000008080808080800000000071
:103F500000C0E0E0E0E0C0C00000000000000000A1
:103F60000000000000000000000000000000000051
:103F70000000000000000000000000000000000041
:103F800000000000000000007EFEFEFEFEFEFE00BF
:103F9000000080FEFEFEFEFEFEFEFC00000000FCB7
:103FA000FEFEFEFEFE3E00000000000000008080DD
:103FB0008080808000000000000000000000000001
:103FC00080F8FEFEFEFEFEFEFEFEF0800000000019
:103FD00000000000000000000080808080808000E1
:103FE0000000000000F8F8F8F8F8F8F80000000009
:103FF000000000000000000000000000E0F0F8FCFD
:10400000FCFEFE7E7E3E3E7E7EFEFCFC78300000A6
:104010000000F8F8F8F8F8F8F800000000000000D8
:104020000000000000000000000000000000000090
:104030000000000000000000000080808080800000
:10404000FFFFFFFFFFFFFF000000030F1F1F1F1FE9
:104050000F0F0000000000000000008080808080C2
:104060008080000000000000000000000000000050
:104070000000000000000000000000000000000040
:104080000000003FFFFFFFFFFFFC00C0FFFFFFFF3E
:104090007FFFFFFFFFFF8000FEFFFFFFFFFF0F001E
:1040A0000000F0F8FEFEFFFF7F1F0F0F1FFFFFFF56
:1040B000FEFCF8C000000000C0FCFFFFFFFF7F0710
:1040C0001FFFFFFFFFFFF88000000000C0F0FCFEB4
:1040D000FFFFFF7F1F1F1F1F3F3F3F0E041F1FFFDC
:1040E000FFFFFFFFFFFF1F1F1F1F0000000000005A
:1040F0000000000000001F7FFFFFFFFFFFFCF8F83B
:10410000F0F0E0E0C1C08000001F1F1FFFFFFFFFB5
:10411000FFFFFF1F1F1F0F000000FFFFFFFFFFFF3C
:1041200000000000FFFFFFFFFFFFFF000000C0F8DE
:10413000FCFEFFFFFF7F1F1F1F3FFFFFFFFFFFFF73
:10414000FF00000000FFFFFFFFFFFFFF000000C0B7
:10415000F8FCFEFFFFFF3F1F1F1F3FFFFFFFFEFC9E
:10416000F8E0000000000000000000000000000077
:1041700000000000000000000000000000000FFF31
:10418000FFFFFFFFFCFFFFFFFF1F0001FFFFFFFF1F
:10419000FFFEFFFFFFFFFF070000001EFFFFFFFF06
:1041A000FFFFDF1F1F1F1F1F1F9F9F1F1F1F0000DD
:1041B000E0FEFFFFFFFFFFFFFCFCFCFDFFFFFFFF3A
:1041C000FFFFFCC00000FFFFFFFFFFFFFF800000BC
:1041D000000000800000000000FFFFFFFFFFFFFF66
:1041E00000000000000000000000000000000000CF
:1041F00080C0C0800101030303070FFFFFFFFFFF23
:10420000FFFF70000000FFFFFFFFFFFFFF00000047
:1042100000000000FFFFFFFFFFFF00000080FFFF26
:10422000FFFFFFFFFF000000FFFFFFFFFFFFFF801A
:1042300000000000FFFFFFFFFFFFFF00000000FF86
:10424000FFFFFFFFFFFF000000FFFFFFFFFFFFFF7B
:104250008000000000FFFFFFFFFFFFFF00000000E5
:10426000000000000000000000000000000000004E
:10427000000000000000000000073F3F3F3F3F3FBD
:104280003F3F0F000000003F3F3F3F3F3F3F3F3F6A
:1042900001000000000001070F1F1F3F3F3F3E3E8F
:1042A0003E3E3F3F1F1F0E00303E3F3F3F3F3F1F00
:1042B00001000000000000033F3F3F3F3F3F3C0044
:1042C0000003070F1F3F3F3F3F3E3E3F3F3F1F1E44
:1042D000080000030F1F3F3F3F3F3F3E3F3F1C187A
:1042E000000000000000000000070F1F1F3F3F3FBD
:1042F0003F3E3E3F3F3F3F1F1F0F070300000000B0
:10430000070F1F3F3F3F3F3E3F3F3F1C00000F1F37
:104310003F3F3F3F3F3E3F1F1F3F3F3F3F3F3F002D
:10432000000000070F1F3F3F3F3F3F3E3F1F1F3F23
:104330003F3F3F3F3F000000003F3F3F3F3F3F3F89
:104340000000000003070F1F3F3F3F3F3E3E3F3F3F
:104350003F1F1F0F030000000000000000000000CE
:10436000000000000000000000000000000000004D
:10437000000000000000000000000000000000003D
:10438000000000000000000000000000000000002D
:10439000000000000000000000000000000000001D
:10494000604900080000002008000000C0010008C5
:104950006849000808000020802B0000DC010008E6
:084960000100000000127A00C2
:040000050800018569
:00000001FF
